:020000040000FA
:0600000016EF07F01200EC
:0608000016EF07F01200E4
:0608080046EF06F01200AD
:06082A000100600E000059
:0808300000020000240000009A
:08083800D9CFE6FFE1CFD9FFA3
:10084000040EE126DE6ADE6ADE6ADD6ADD52DD5212
:10085000FD0EDBCF00F0FE0EDBCF01F0026A036A73
:1008600001AE02D002680368D9CFE9FFDACFEAFF10
:10087000030EEB500318E8AE02D0033408D000504A
:10088000EE5C0150EE580250EE580350EE580FE265
:100890000C0EE66EF6EC06F0E552D9CFE9FFDACFA2
:1008A000EAFFEE2A000EEE22EE22EE22D1D7040E4F
:1008B000E15C02E2E16AE552E16EE552E7CFD9FF81
:1008C00012000F0EC16E070EB46E936A300E926E58
:1008D0000F0E946EF19E1200D9CFE6FFE1CFD9FF43
:1008E000020EE1268250020B01E0010E080DF3CF4B
:1008F00002F08250010B040DF3CF01F08050200B69
:1009000001E0010EE824006E8050100B01E0010EA2
:10091000002401240224DE6EDD6ADECF00F0DDCF8C
:1009200001F000C0F3FF01C0F4FF020EE15C03E23E
:1009300000D0E16AE552E16EE552E7CFD9FF12003F
:100940008092320EE66E24EC07F0E5528084320E7F
:10095000E66E24EC07F0E5528094320EE66E24EC4D
:1009600007F0E55212008082320EE66E24EC07F0AA
:10097000E5528084320EE66E24EC07F0E552809456
:10098000320EE66E24EC07F0E5521200380E816E4E
:10099000D7DF320EE66EE66A4FDFE552E552010E12
:1009A000816ECEDF320EE66EE66A46DFE552E55234
:1009B0000D0E816EC5DF320EE66EE66A3DDFE55252
:1009C000E552060E816EBCDF320EE66EE66A34DF5B
:1009D000E552E5521200010E816EB2DF0A0EE66E9C
:1009E000E66A2ADFE552E5521200D9CFE6FFE1CFF1
:1009F000D9FF020E816EA4DF0A0EE66EE66A1CDFE6
:100A0000E552E552FD0EDBCFE6FFFE0EDB50280D72
:100A1000F350E552E724E76EFE0EE7CFDBFFFD0E55
:100A2000DB6AFE0EDB50F36EFD0EDBCFF4FFF350FE
:100A3000F45C0BE2140E816E83DF320EE66E24EC62
:100A400007F0E552FD0EDB2AECD7E552E7CFD9FFE0
:100A50001200D9CFE6FFE1CFD9FFFE0EDB50816E49
:100A600082DF320EE66E24EC07F0E552E552E7CF66
:100A7000D9FF1200D9CFE6FFE1CFD9FFFD0EDBCFC2
:100A8000E9FFFE0EDBCFEAFFEF500EE0FD0EDBCFFD
:100A9000E9FFDB2AFE0EDBCFEAFF01E3DB2AEF50A2
:100AA000E66ED7DFE552EAD7E552E7CFD9FF12006D
:100AB0000201286B300E926EF00E936EEF0E246FD3
:100AC00024C281FF040E256F2551000821E2245124
:100AD000FE0BE842246F24C281FF050EE66EE66A33
:100AE000ABDEE552E5528150100B09E08150200B3E
:100AF00006E08150400B03E08150800B01E10AD8F1
:100B00000201280502E1295104D02505256FDCD713
:100B1000CFD71200F00E936E81CF27F20201271576
:100B2000266F0F0E2415246F24512611246F81CFB8
:100B300027F2F00E2715266FF00E265D01E0F7D79D
:100B4000936A06D82AC229F20201010E286F120008
:100B500002012B6B100E2B5D14E22B51EA6A000F81
:100B6000E96E020EEA22EF50245D08E12B51EA6A99
:100B7000100FE96E020EEA22EFCF2AF22B292B6F1B
:100B8000E9D72AC281FF640EE66EE66A55DEE552B9
:100B9000E552120002012C6B070E2C5D1DE288DF6E
:100BA00002012D6F2C51EA6A2E0FE96E020EEA2225
:100BB0002DC2EFFF2C51EA6A2E0FE96E020EEA22D7
:100BC000EF50460802E108D004D02DC2E6FF41DF15
:100BD000E55202012C2BE0D72C51EA6A2E0FE96E68
:100BE000020EEA22EF6A120002012C6B070E2C5D46
:100BF00016E22C51EA6A2E0FE96E020EEA22EF503D
:100C0000E66E27DFE55202012C29EA6A2E0FE96E13
:100C1000020EEA22EF5001E102D02C2BE7D712009E
:100C2000D9CFE6FFE1CFD9FFE652F250800B01E0C9
:100C3000010EDF6EF29EA69EA69CA684FE0EDB50E1
:100C4000A96EFD0EDB50A86E550EA76EAA0EA76EFC
:100C5000A682A6B2FED7A694DF50E8B0F28EE8A036
:100C6000F29EE552E552E7CFD9FF1200D9CFE6FF59
:100C7000E1CFD9FFA69CA69EFE0EDB50A96EA680F2
:100C8000A85000D0E552E7CFD9FF1200DACFE4FF39
:100C9000E2CFDAFFE65202013907000E3A5BD89044
:100CA0003A51000A08E6000E375D000E3859010E71
:100CB0003959000E3A5909E21B0E3827B70E39236D
:100CC000000E3A230201202B2123F294E552E5CFB6
:100CD000DAFF1100F6DD816A0201376B1B0E386FF7
:100CE000B70E396F3A6B9F0EE66EDAEC06F0E552FE
:100CF000F28E02012251201902E12351211909E04B
:100D000020C222F221C223F281A002D0819001D020
:060D10008180EFD7120004
:0A0D16002A0EF66E080EF76E000EAE
:100D2000F86E00010900F550656F0900F550666F17
:100D300003E1656701D03DD00900F550606F0900FF
:100D4000F550616F0900F550626F09000900F55018
:100D5000E96E0900F550EA6E090009000900F55036
:100D6000636F0900F550646F09000900F6CF67F062
:100D7000F7CF68F0F8CF69F060C0F6FF61C0F7FF09
:100D800062C0F8FF0001635302E1645307E0090009
:100D9000F550EE6E6307F8E26407F9D767C0F6FF17
:100DA00068C0F7FF69C0F8FF00016507000E665BC9
:040DB000BFD7120097
:0C0DB400D9CFE6FFDACFE6FFE1CFD9FF90
:100DC000E2CFDAFFFD0EDB507F0BD56ED76AD66A15
:100DD000F294FD0EDBAE02D0F28A01D0F29AD58EEB
:0C0DE000E552E5CFDAFFE7CFD9FF1200A3
:040DEC00FF0EE350C3
:100DF000066E480E01D04C0EE76EE72EFED7E76A6E
:0C0E0000E72EFED7062EF7D700001200E8
:040E0C00000EF36E73
:100E100000EE00F0080E01D81200EA6002D0EE6A7F
:0C0E2000FCD7F350E9601200EE6AFCD72A
:040E2C0012EE40F092
:100E300022EE40F0F86A059C8BEC06F02FEC07F0F0
:080E40006AEC06F0FBD712007A
:080E4800FF0EE350E84E12001A
:0E0E5000000000D000D000D0E82EFAD712002B
:020E5E00120080
:100E6000EEEDEBE7DEDDDBD7BEBDBBB77E7D7B778E
:100E700030313233343536373839414243444546D0
:040E8000000000006E
:00000001FF
